BL51 BANKED LINKER/LOCATER V6.22                                                        08/15/2017  09:10:53  PAGE 1


BL51 BANKED LINKER/LOCATER V6.22, INVOKED BY:
C:\KEIL\C51\BIN\BL51.EXE STARTUP.obj, Main.obj, USART.obj TO 串口通信测试 CODE (0X0000-0X0FFF)


MEMORY MODEL: SMALL


INPUT MODULES INCLUDED:
  STARTUP.obj (?C_STARTUP)
  Main.obj (MAIN)
  USART.obj (USART)
  C:\KEIL\C51\LIB\C51S.LIB (?C?CLDPTR)
  C:\KEIL\C51\LIB\C51S.LIB (?C?CSTPTR)


LINK MAP OF MODULE:  串口通信测试 (?C_STARTUP)


            TYPE    BASE      LENGTH    RELOCATION   SEGMENT NAME
            -----------------------------------------------------

            * * * * * * *   D A T A   M E M O R Y   * * * * * * *
            REG     0000H     0008H     ABSOLUTE     "REG BANK 0"
            DATA    0008H     0003H     UNIT         ?DT?USART
            DATA    000BH     0001H     UNIT         _DATA_GROUP_
            IDATA   000CH     0001H     UNIT         ?STACK

            * * * * * * *   C O D E   M E M O R Y   * * * * * * *
            CODE    0000H     0003H     ABSOLUTE     
            CODE    0003H     0019H     UNIT         ?PR?INITSERIALPORT?USART
                    001CH     0007H                  *** GAP ***
            CODE    0023H     0003H     ABSOLUTE     
            CODE    0026H     002DH     UNIT         ?PR?SERIALPORTINTE?USART
            CODE    0053H     002BH     UNIT         ?C?LIB_CODE
            CODE    007EH     0013H     UNIT         ?PR?_SENDSTRING?USART
            CODE    0091H     0010H     UNIT         ?PR?MAIN?MAIN
            CODE    00A1H     000CH     UNIT         ?C_C51STARTUP
            CODE    00ADH     0008H     UNIT         ?PR?RECEIVEBYTE?USART
            CODE    00B5H     0008H     UNIT         ?PR?_SENDBYTE?USART



OVERLAY MAP OF MODULE:   串口通信测试 (?C_STARTUP)


SEGMENT                            DATA_GROUP 
  +--> CALLED SEGMENT            START    LENGTH
------------------------------------------------
?C_C51STARTUP                    -----    -----
  +--> ?PR?MAIN?MAIN

?PR?MAIN?MAIN                    000BH    0001H
  +--> ?PR?INITSERIALPORT?USART
  +--> ?PR?RECEIVEBYTE?USART
  +--> ?PR?_SENDBYTE?USART



BL51 BANKED LINKER/LOCATER V6.22                                                      08/15/2017  09:10:53  PAGE 2


SYMBOL TABLE OF MODULE:  串口通信测试 (?C_STARTUP)

  VALUE           TYPE          NAME
  ----------------------------------

  -------         MODULE        ?C_STARTUP
  C:00A1H         SEGMENT       ?C_C51STARTUP
  I:000CH         SEGMENT       ?STACK
  C:0000H         PUBLIC        ?C_STARTUP
  D:00E0H         SYMBOL        ACC
  D:00F0H         SYMBOL        B
  D:0083H         SYMBOL        DPH
  D:0082H         SYMBOL        DPL
  N:0000H         SYMBOL        IBPSTACK
  N:0100H         SYMBOL        IBPSTACKTOP
  N:0080H         SYMBOL        IDATALEN
  C:00A4H         SYMBOL        IDATALOOP
  N:0000H         SYMBOL        PBPSTACK
  N:0100H         SYMBOL        PBPSTACKTOP
  N:0000H         SYMBOL        PDATALEN
  N:0000H         SYMBOL        PDATASTART
  N:0000H         SYMBOL        PPAGE
  N:0000H         SYMBOL        PPAGEENABLE
  D:00A0H         SYMBOL        PPAGE_SFR
  D:0081H         SYMBOL        SP
  C:00A1H         SYMBOL        STARTUP1
  N:0000H         SYMBOL        XBPSTACK
  N:0000H         SYMBOL        XBPSTACKTOP
  N:0000H         SYMBOL        XDATALEN
  N:0000H         SYMBOL        XDATASTART
  C:0000H         LINE#         126
  C:00A1H         LINE#         133
  C:00A3H         LINE#         134
  C:00A4H         LINE#         135
  C:00A5H         LINE#         136
  C:00A7H         LINE#         185
  C:00AAH         LINE#         196
  -------         ENDMOD        ?C_STARTUP

  -------         MODULE        MAIN
  C:0000H         SYMBOL        _ICE_DUMMY_
  D:0080H         PUBLIC        P0
  D:0090H         PUBLIC        P1
  D:00A0H         PUBLIC        P2
  D:00B0H         PUBLIC        P3
  D:00C0H         PUBLIC        P4
  D:00C8H         PUBLIC        P5
  D:00E8H         PUBLIC        P6
  D:00F8H         PUBLIC        P7
  D:00A8H         PUBLIC        IE
  D:00B8H         PUBLIC        IP
  D:00D8H         PUBLIC        CCON
  C:0091H         PUBLIC        main
  D:0098H         PUBLIC        SCON
  D:0088H         PUBLIC        TCON
  D:00D0H         PUBLIC        PSW
  -------         PROC          MAIN
BL51 BANKED LINKER/LOCATER V6.22                                                      08/15/2017  09:10:53  PAGE 3


  -------         DO            
  D:000BH         SYMBOL        rdata
  -------         ENDDO         
  C:0091H         LINE#         30
  C:0091H         LINE#         31
  C:0091H         LINE#         32
  C:0094H         LINE#         33
  C:0097H         LINE#         35
  C:0097H         LINE#         36
  C:0097H         LINE#         37
  C:009CH         LINE#         38
  C:009FH         LINE#         39
  -------         ENDPROC       MAIN
  -------         ENDMOD        MAIN

  -------         MODULE        USART
  C:0000H         SYMBOL        _ICE_DUMMY_
  D:0080H         PUBLIC        P0
  D:0090H         PUBLIC        P1
  D:00A0H         PUBLIC        P2
  D:00B0H         PUBLIC        P3
  D:00C0H         PUBLIC        P4
  D:00C8H         PUBLIC        P5
  D:00E8H         PUBLIC        P6
  D:00F8H         PUBLIC        P7
  C:007EH         PUBLIC        _SendString
  D:00A8H         PUBLIC        IE
  D:0008H         PUBLIC        pchar
  D:00B8H         PUBLIC        IP
  B:0098H.0       PUBLIC        RI
  B:0098H.1       PUBLIC        TI
  C:0026H         PUBLIC        SerialPortInte
  C:00B5H         PUBLIC        _SendByte
  C:0003H         PUBLIC        InitSerialPort
  D:00D8H         PUBLIC        CCON
  D:0099H         PUBLIC        SBUF
  D:0098H         PUBLIC        SCON
  D:0088H         PUBLIC        TCON
  D:008EH         PUBLIC        AUXR
  D:00D6H         PUBLIC        T2H
  B:0098H.7       PUBLIC        SM0
  B:0098H.6       PUBLIC        SM1
  D:00D7H         PUBLIC        T2L
  C:00ADH         PUBLIC        ReceiveByte
  B:0098H.4       PUBLIC        REN
  D:00D0H         PUBLIC        PSW
  -------         PROC          INITSERIALPORT
  C:0003H         LINE#         35
  C:0003H         LINE#         36
  C:0003H         LINE#         37
  C:0006H         LINE#         38
  C:0009H         LINE#         39
  C:000CH         LINE#         40
  C:000FH         LINE#         41
  C:0012H         LINE#         42
  C:0015H         LINE#         44
  C:0017H         LINE#         45
BL51 BANKED LINKER/LOCATER V6.22                                                      08/15/2017  09:10:53  PAGE 4


  C:0019H         LINE#         46
  C:001BH         LINE#         47
  -------         ENDPROC       INITSERIALPORT
  -------         PROC          RECEIVEBYTE
  -------         DO            
  D:0007H         SYMBOL        rbyte
  -------         ENDDO         
  C:00ADH         LINE#         52
  C:00ADH         LINE#         53
  C:00ADH         LINE#         55
  C:00B0H         LINE#         56
  C:00B2H         LINE#         57
  C:00B4H         LINE#         58
  C:00B4H         LINE#         59
  -------         ENDPROC       RECEIVEBYTE
  -------         PROC          _SENDBYTE
  D:0007H         SYMBOL        sbyte
  C:00B5H         LINE#         64
  C:00B5H         LINE#         65
  C:00B5H         LINE#         66
  C:00B7H         LINE#         67
  C:00BAH         LINE#         68
  C:00BCH         LINE#         69
  -------         ENDPROC       _SENDBYTE
  -------         PROC          _SENDSTRING
  D:0001H         SYMBOL        pstr
  C:007EH         LINE#         74
  C:007EH         LINE#         75
  C:007EH         LINE#         76
  C:0084H         LINE#         77
  C:0084H         LINE#         78
  C:0087H         LINE#         79
  C:008EH         LINE#         80
  C:0090H         LINE#         81
  -------         ENDPROC       _SENDSTRING
  -------         PROC          SERIALPORTINTE
  C:0026H         LINE#         86
  C:0037H         LINE#         88
  C:0039H         LINE#         89
  C:0044H         LINE#         90
  -------         ENDPROC       SERIALPORTINTE
  -------         ENDMOD        USART

  -------         MODULE        ?C?CLDPTR
  C:0053H         PUBLIC        ?C?CLDPTR
  -------         ENDMOD        ?C?CLDPTR

  -------         MODULE        ?C?CSTPTR
  C:006CH         PUBLIC        ?C?CSTPTR
  -------         ENDMOD        ?C?CSTPTR

*** WARNING L16: UNCALLED SEGMENT, IGNORED FOR OVERLAY PROCESS
    SEGMENT: ?PR?_SENDSTRING?USART

Program Size: data=13.0 xdata=0 code=182
LINK/LOCATE RUN COMPLETE.  1 WARNING(S),  0 ERROR(S)
